 imx_xvc

 Timestamp is 4fb05c73 (Mon May 14 13:14:27 2012)

 Preferred load address is 10000000

 Start         Length     Name                   Class
 0001:00000000 00000004H .CRT$XCA                CODE
 0001:00000004 00000004H .CRT$XCZ                CODE
 0001:00000008 00000004H .CRT$XIA                CODE
 0001:0000000c 00000004H .CRT$XIZ                CODE
 0001:00000010 00000004H .CRT$XPA                CODE
 0001:00000014 00000004H .CRT$XPZ                CODE
 0001:00000018 00000004H .CRT$XTA                CODE
 0001:0000001c 00000004H .CRT$XTZ                CODE
 0001:00000020 00002594H .rdata                  CODE
 0001:000025b4 00000024H .rdata$debug            CODE
 0001:000025d8 00006af8H .text                   CODE
 0001:000090d0 0000001cH .xdata                  CODE
 0001:000090ec 0000003cH .idata$2                CODE
 0001:00009128 00000014H .idata$3                CODE
 0001:0000913c 000000e4H .idata$4                CODE
 0001:00009220 00000068H .idata$6                CODE
 0001:00009290 00000104H .edata                  CODE
 0002:00000000 000000e4H .idata$5                DATA
 0002:000000e8 00000450H .data                   DATA
 0002:00000538 00000020H .bss                    DATA
 0003:00000000 00000278H .pdata                  DATA

  Address         Publics by Value              Rva+Base       Lib:Object

 0000:00000000       ___safe_se_handler_count   00000000     <absolute>
 0000:00000000       ___safe_se_handler_table   00000000     <absolute>
 0001:00000000       __xc_a                     10001000     corelib0:crt0init.obj
 0001:00000004       __xc_z                     10001004     corelib0:crt0init.obj
 0001:00000008       __xi_a                     10001008     corelib0:crt0init.obj
 0001:0000000c       __xi_z                     1000100c     corelib0:crt0init.obj
 0001:00000010       __xp_a                     10001010     corelib0:crt0init.obj
 0001:00000014       __xp_z                     10001014     corelib0:crt0init.obj
 0001:00000018       __xt_a                     10001018     corelib0:crt0init.obj
 0001:0000001c       __xt_z                     1000101c     corelib0:crt0init.obj
 0001:000000d0       ??_C@_1DE@KOFCAGHF@?$AA?7?$AAU?$AAS?$AAB?$AA_?$AAO?$AAT?$AAG?$AA_?$AAM?$AAI?$AAR?$AAR?$AAO?$AAR?$AA?$CI?$AA?$CF?$AAx?$AAh?$AA?$CJ?$AA?$DN?$AA?$CF?$AAx?$AA?$AN?$AA?6?$AA?$AA@ 100010d0     hwinit.obj
 0001:00000104       ??_C@_1CI@PDMEMNIO@?$AA?7?$AAU?$AAS?$AAB?$AA_?$AAC?$AAT?$AAR?$AAL?$AA?$CI?$AA?$CF?$AAx?$AAh?$AA?$CJ?$AA?$DN?$AA?$CF?$AAx?$AA?$AN?$AA?6?$AA?$AA@ 10001104     hwinit.obj
 0001:0000012c       ??_C@_1CM@JDNJIAPD@?$AA?7?$AAE?$AAN?$AAD?$AAP?$AAT?$AAC?$AAT?$AAR?$AAL?$AA0?$AA?$CI?$AA?$CF?$AAx?$AAh?$AA?$CJ?$AA?$DN?$AA?$CF?$AAx?$AA?$AN?$AA?6?$AA?$AA@ 1000112c     hwinit.obj
 0001:00000158       ??_C@_1DC@KJHNCNIC@?$AA?7?$AAE?$AAN?$AAD?$AAP?$AAT?$AAC?$AAO?$AAM?$AAP?$AAL?$AAE?$AAT?$AAE?$AA?$CI?$AA?$CF?$AAx?$AAh?$AA?$CJ?$AA?$DN?$AA?$CF?$AAx?$AA?$AN?$AA?6?$AA?$AA@ 10001158     hwinit.obj
 0001:0000018c       ??_C@_1CO@OOCOBPDB@?$AA?7?$AAE?$AAN?$AAD?$AAP?$AAT?$AAS?$AAT?$AAA?$AAT?$AAU?$AAS?$AA?$CI?$AA?$CF?$AAx?$AAh?$AA?$CJ?$AA?$DN?$AA?$CF?$AAx?$AA?$AN?$AA?6?$AA?$AA@ 1000118c     hwinit.obj
 0001:000001bc       ??_C@_1CM@NMOAEIN@?$AA?7?$AAE?$AAN?$AAD?$AAP?$AAT?$AAF?$AAL?$AAU?$AAS?$AAH?$AA?$CI?$AA?$CF?$AAx?$AAh?$AA?$CJ?$AA?$DN?$AA?$CF?$AAx?$AA?$AN?$AA?6?$AA?$AA@ 100011bc     hwinit.obj
 0001:000001e8       ??_C@_1CM@HCKMLEJH@?$AA?7?$AAE?$AAN?$AAD?$AAP?$AAT?$AAP?$AAR?$AAI?$AAM?$AAE?$AA?$CI?$AA?$CF?$AAx?$AAh?$AA?$CJ?$AA?$DN?$AA?$CF?$AAx?$AA?$AN?$AA?6?$AA?$AA@ 100011e8     hwinit.obj
 0001:00000214       ??_C@_1DE@KNPJONMF@?$AA?7?$AAE?$AAN?$AAD?$AAP?$AAT?$AAS?$AAE?$AAT?$AAU?$AAP?$AAS?$AAT?$AAA?$AAT?$AA?$CI?$AA?$CF?$AAx?$AAh?$AA?$CJ?$AA?$DN?$AA?$CF?$AAx?$AA?$AN?$AA?6?$AA?$AA@ 10001214     hwinit.obj
 0001:00000248       ??_C@_1DC@HGNFDDAA@?$AA?7?$AAA?$AAS?$AAY?$AAN?$AAC?$AAL?$AAI?$AAS?$AAT?$AAA?$AAD?$AAD?$AAR?$AA?$CI?$AA?$CF?$AAx?$AAh?$AA?$CJ?$AA?$DN?$AA?$CF?$AAx?$AA?$AN?$AA?6?$AA?$AA@ 10001248     hwinit.obj
 0001:00000280       ??_C@_1EI@NFAOHDEB@?$AA?7?$AAA?$AAd?$AAd?$AAr?$AAe?$AAs?$AAs?$AA?5?$AAo?$AAf?$AA?5?$AAA?$AAS?$AAY?$AAN?$AAC?$AAL?$AAI?$AAS?$AAT?$AAA?$AAD?$AAD?$AAR?$AA?5?$AAa?$AAt?$AA?5?$AA0?$AAx?$AA?$CF@ 10001280     hwinit.obj
 0001:000002c8       ??_C@_1DC@LGOMINDC@?$AA?7?$AA?$CK?$AA?$CK?$AA?$CK?$AA?$CK?$AA?$CK?$AA?$CK?$AA?$CK?$AA?$CK?$AA?$CK?$AA?$CK?$AA?$CK?$AA?$CK?$AA?$CK?$AA?$CK?$AA?$CK?$AA?$CK?$AA?$CK?$AA?$CK?$AA?$CK?$AA?$CK?$AA?$CK?$AA?$AN?$AA?6?$AA?$AA@ 100012c8     hwinit.obj
 0001:000002fc       ??_C@_1DC@CMAILMML@?$AA?7?$AAU?$AAL?$AAP?$AAI?$AA_?$AAV?$AAI?$AAE?$AAW?$AAP?$AAO?$AAR?$AAT?$AA?$CI?$AA?$CF?$AAx?$AAh?$AA?$CJ?$AA?$DN?$AA?$CF?$AAx?$AA?$AN?$AA?6?$AA?$AA@ 100012fc     hwinit.obj
 0001:00000330       ??_C@_1CG@GAIKAENJ@?$AA?7?$AAU?$AAS?$AAB?$AAM?$AAO?$AAD?$AAE?$AA?$CI?$AA?$CF?$AAx?$AAh?$AA?$CJ?$AA?$DN?$AA?$CF?$AAx?$AA?$AN?$AA?6?$AA?$AA@ 10001330     hwinit.obj
 0001:00000358       ??_C@_1CC@CBNJLNBD@?$AA?7?$AAO?$AAT?$AAG?$AAS?$AAC?$AA?$CI?$AA?$CF?$AAx?$AAh?$AA?$CJ?$AA?$DN?$AA?$CF?$AAx?$AA?$AN?$AA?6?$AA?$AA@ 10001358     hwinit.obj
 0001:0000037c       ??_C@_1CK@FFFOFLFA@?$AA?7?$AAP?$AAO?$AAR?$AAT?$AAS?$AAC?$AA?$CI?$AA?$CF?$AAx?$AAh?$AA?$CJ?$AA?$FL?$AA0?$AA?$FN?$AA?$DN?$AA?$CF?$AAx?$AA?$AN?$AA?6?$AA?$AA@ 1000137c     hwinit.obj
 0001:000003a8       ??_C@_1CG@HEJNGGNG@?$AA?7?$AAU?$AAS?$AAB?$AAI?$AAN?$AAT?$AAR?$AA?$CI?$AA?$CF?$AAx?$AAh?$AA?$CJ?$AA?$DN?$AA?$CF?$AAx?$AA?$AN?$AA?6?$AA?$AA@ 100013a8     hwinit.obj
 0001:000003d0       ??_C@_1CE@PNIDKFEL@?$AA?7?$AAU?$AAS?$AAB?$AAS?$AAT?$AAS?$AA?$CI?$AA?$CF?$AAx?$AAh?$AA?$CJ?$AA?$DN?$AA?$CF?$AAx?$AA?$AN?$AA?6?$AA?$AA@ 100013d0     hwinit.obj
 0001:000003f4       ??_C@_1CE@LAMJOMIC@?$AA?7?$AAU?$AAS?$AAB?$AAC?$AAM?$AAD?$AA?$CI?$AA?$CF?$AAx?$AAh?$AA?$CJ?$AA?$DN?$AA?$CF?$AAx?$AA?$AN?$AA?6?$AA?$AA@ 100013f4     hwinit.obj
 0001:00000418       ??_C@_1CK@MJMJCCJH@?$AA?7?$AAD?$AAC?$AAC?$AAP?$AAA?$AAR?$AAA?$AAM?$AAS?$AA?$CI?$AA?$CF?$AAx?$AAh?$AA?$CJ?$AA?$DN?$AA?$CF?$AAx?$AA?$AN?$AA?6?$AA?$AA@ 10001418     hwinit.obj
 0001:00000444       ??_C@_1CM@OEHCBFKM@?$AA?7?$AAD?$AAC?$AAI?$AAV?$AAE?$AAR?$AAS?$AAI?$AAO?$AAN?$AA?$CI?$AA?$CF?$AAx?$AAh?$AA?$CJ?$AA?$DN?$AA?$CF?$AAx?$AA?$AN?$AA?6?$AA?$AA@ 10001444     hwinit.obj
 0001:00000470       ??_C@_1CK@GDDLOALH@?$AA?7?$AAH?$AAC?$AAC?$AAP?$AAA?$AAR?$AAA?$AAM?$AAS?$AA?$CI?$AA?$CF?$AAx?$AAh?$AA?$CJ?$AA?$DN?$AA?$CF?$AAx?$AA?$AN?$AA?6?$AA?$AA@ 10001470     hwinit.obj
 0001:0000049c       ??_C@_1CK@ICHKICOL@?$AA?7?$AAH?$AAC?$AAS?$AAP?$AAA?$AAR?$AAA?$AAM?$AAS?$AA?$CI?$AA?$CF?$AAx?$AAh?$AA?$CJ?$AA?$DN?$AA?$CF?$AAx?$AA?$AN?$AA?6?$AA?$AA@ 1000149c     hwinit.obj
 0001:000004c8       ??_C@_1CM@EJMDIGA@?$AA?7?$AAH?$AAC?$AAI?$AAV?$AAE?$AAR?$AAS?$AAI?$AAO?$AAN?$AA?$CI?$AA?$CF?$AAx?$AAh?$AA?$CJ?$AA?$DN?$AA?$CF?$AAx?$AA?$AN?$AA?6?$AA?$AA@ 100014c8     hwinit.obj
 0001:000004f4       ??_C@_1CK@BONIGHNC@?$AA?7?$AAC?$AAA?$AAP?$AAL?$AAE?$AAN?$AAG?$AAT?$AAH?$AA?$CI?$AA?$CF?$AAx?$AAh?$AA?$CJ?$AA?$DN?$AA?$CF?$AAx?$AA?$AN?$AA?6?$AA?$AA@ 100014f4     hwinit.obj
 0001:00000520       ??_C@_1CG@HBIIJHPE@?$AA?7?$AAH?$AAW?$AAR?$AAX?$AAB?$AAU?$AAF?$AA?$CI?$AA?$CF?$AAx?$AAh?$AA?$CJ?$AA?$DN?$AA?$CF?$AAx?$AA?$AN?$AA?6?$AA?$AA@ 10001520     hwinit.obj
 0001:00000548       ??_C@_1CG@DIMHIAML@?$AA?7?$AAH?$AAW?$AAT?$AAX?$AAB?$AAU?$AAF?$AA?$CI?$AA?$CF?$AAx?$AAh?$AA?$CJ?$AA?$DN?$AA?$CF?$AAx?$AA?$AN?$AA?6?$AA?$AA@ 10001548     hwinit.obj
 0001:00000570       ??_C@_1CI@LAAAOKFK@?$AA?7?$AAH?$AAW?$AAD?$AAE?$AAV?$AAI?$AAC?$AAE?$AA?$CI?$AA?$CF?$AAx?$AAh?$AA?$CJ?$AA?$DN?$AA?$CF?$AAx?$AA?$AN?$AA?6?$AA?$AA@ 10001570     hwinit.obj
 0001:00000598       ??_C@_1CE@FJBMGFNB@?$AA?7?$AAH?$AAW?$AAH?$AAO?$AAS?$AAT?$AA?$CI?$AA?$CF?$AAx?$AAh?$AA?$CJ?$AA?$DN?$AA?$CF?$AAx?$AA?$AN?$AA?6?$AA?$AA@ 10001598     hwinit.obj
 0001:000005bc       ??_C@_1CK@ECFJBANB@?$AA?7?$AAH?$AAW?$AAG?$AAE?$AAN?$AAE?$AAR?$AAA?$AAL?$AA?$CI?$AA?$CF?$AAx?$AAh?$AA?$CJ?$AA?$DN?$AA?$CF?$AAx?$AA?$AN?$AA?6?$AA?$AA@ 100015bc     hwinit.obj
 0001:000005e8       ??_C@_1BM@DCDGAICD@?$AA?7?$AAI?$AAD?$AA?$CI?$AA?$CF?$AAx?$AAh?$AA?$CJ?$AA?$DN?$AA?$CF?$AAx?$AA?$AN?$AA?6?$AA?$AA@ 100015e8     hwinit.obj
 0001:00000604       ??_C@_1CA@JNECBFDG@?$AAD?$AAu?$AAm?$AAp?$AA?5?$AAO?$AAT?$AAG?$AA?5?$AAR?$AAe?$AAg?$AAs?$AA?$AN?$AA?6?$AA?$AA@ 10001604     hwinit.obj
 0001:00000624       ??_C@_1DM@PINNGIJL@?$AA?7?$AA?7?$AA?7?$AAS?$AAe?$AAr?$AAi?$AAa?$AAl?$AA?1?$AA1?$AA?4?$AA1?$AA?5?$AAP?$AAH?$AAY?$AA?5?$AA?$CI?$AAF?$AAS?$AA?5?$AAO?$AAn?$AAl?$AAy?$AA?$CJ?$AA?$AN?$AA?6?$AA?$AA@ 10001624     hwinit.obj
 0001:00000660       ??_C@_1BE@OHMKGMAA@?$AA?7?$AA?7?$AA?7?$AAU?$AAL?$AAP?$AAI?$AA?$AN?$AA?6?$AA?$AA@ 10001660     hwinit.obj
 0001:00000674       ??_C@_1CK@JDCKMGFE@?$AA?7?$AA?7?$AA?7?$AAP?$AAh?$AAi?$AAl?$AAi?$AAp?$AAs?$AA?5?$AAC?$AAl?$AAa?$AAs?$AAs?$AAi?$AAc?$AA?$AN?$AA?6?$AA?$AA@ 10001674     hwinit.obj
 0001:000006a0       ??_C@_1CA@GIFIBBC@?$AA?7?$AA?7?$AA?7?$AAU?$AAT?$AAM?$AAI?$AA?1?$AAU?$AAT?$AAM?$AAI?$AA?$CL?$AA?$AN?$AA?6?$AA?$AA@ 100016a0     hwinit.obj
 0001:000006c0       ??_C@_1EG@GEPPEHI@?$AA?7?$AA?7?$AAP?$AAa?$AAr?$AAa?$AAl?$AAl?$AAe?$AAl?$AA?5?$AAT?$AAr?$AAa?$AAn?$AAs?$AAc?$AAe?$AAi?$AAv?$AAe?$AAr?$AA?5?$AAS?$AAe?$AAl?$AAe?$AAc?$AAt?$AA?3?$AA?$CF?$AAx@ 100016c0     hwinit.obj
 0001:00000708       ??_C@_1DO@GOALHOBG@?$AA?7?$AA?7?$AAS?$AAe?$AAr?$AAi?$AAa?$AAl?$AA?5?$AAT?$AAr?$AAa?$AAn?$AAs?$AAc?$AAe?$AAi?$AAv?$AAe?$AAr?$AA?5?$AAS?$AAe?$AAl?$AAe?$AAc?$AAt?$AA?5?$AA?$AN?$AA?6?$AA?$AA@ 10001708     hwinit.obj
 0001:00000748       ??_C@_1BI@PMFMKPBN@?$AA?7?$AA?7?$AA?7?$AA8?$AA?5?$AAb?$AAi?$AAt?$AAs?$AA?$AN?$AA?6?$AA?$AA@ 10001748     hwinit.obj
 0001:00000760       ??_C@_1BK@DMIJGPDB@?$AA?7?$AA?7?$AA?7?$AA1?$AA6?$AA?5?$AAb?$AAi?$AAt?$AAs?$AA?$AN?$AA?6?$AA?$AA@ 10001760     hwinit.obj
 0001:00000780       ??_C@_1EE@PJPHJMEN@?$AA?7?$AA?7?$AAP?$AAa?$AAr?$AAa?$AAl?$AAl?$AAe?$AAl?$AA?5?$AAT?$AAr?$AAa?$AAn?$AAs?$AAc?$AAe?$AAi?$AAv?$AAe?$AAr?$AA?5?$AAW?$AAi?$AAd?$AAt?$AAh?$AA?3?$AA?$CF?$AAx?$AA?9@ 10001780     hwinit.obj
 0001:000007c4       ??_C@_1CA@CFDEDDEG@?$AA?7?$AA?7?$AA?7?$AAH?$AAi?$AAg?$AAh?$AA?5?$AAS?$AAp?$AAe?$AAe?$AAd?$AA?$AN?$AA?6?$AA?$AA@ 100017c4     hwinit.obj
 0001:000007e4       ??_C@_1BO@DONMFABC@?$AA?7?$AA?7?$AA?7?$AAL?$AAo?$AAw?$AA?5?$AAS?$AAp?$AAe?$AAe?$AAd?$AA?$AN?$AA?6?$AA?$AA@ 100017e4     hwinit.obj
 0001:00000804       ??_C@_1CA@EFHFHOIO@?$AA?7?$AA?7?$AA?7?$AAF?$AAu?$AAl?$AAl?$AA?5?$AAS?$AAp?$AAe?$AAe?$AAd?$AA?$AN?$AA?6?$AA?$AA@ 10001804     hwinit.obj
 0001:00000824       ??_C@_1CG@DLDJDNPN@?$AA?7?$AA?7?$AAP?$AAo?$AAr?$AAt?$AA?5?$AAS?$AAp?$AAe?$AAe?$AAd?$AA?3?$AA?5?$AA?$CF?$AAx?$AA?9?$AA?$DO?$AA?$AA@ 10001824     hwinit.obj
 0001:00000850       ??_C@_1EG@FLKCNOK@?$AA?7?$AA?7?$AAP?$AAo?$AAr?$AAt?$AA?5?$AAF?$AAo?$AAr?$AAc?$AAe?$AA?5?$AAF?$AAu?$AAl?$AAl?$AA?5?$AAS?$AAp?$AAe?$AAe?$AAd?$AA?5?$AAC?$AAo?$AAn?$AAn?$AAe?$AAc?$AAt?$AA?5@ 10001850     hwinit.obj
 0001:00000898       ??_C@_1GI@HKEGLKNC@?$AA?7?$AA?7?$AAP?$AAH?$AAY?$AA?5?$AAL?$AAo?$AAw?$AA?5?$AAP?$AAo?$AAw?$AAe?$AAr?$AA?5?$AAS?$AAu?$AAs?$AAp?$AAe?$AAn?$AAd?$AA?5?$AA?9?$AA?5?$AAC?$AAl?$AAo?$AAc?$AAk?$AA?5@ 10001898     hwinit.obj
 0001:00000900       ??_C@_1FE@PECIMICA@?$AA?7?$AA?7?$AAW?$AAa?$AAk?$AAe?$AA?5?$AAo?$AAn?$AA?5?$AAO?$AAv?$AAe?$AAr?$AA?9?$AAc?$AAu?$AAr?$AAr?$AAe?$AAn?$AAt?$AA?5?$AAE?$AAn?$AAa?$AAb?$AAl?$AAe?$AA?5?$AA?$CI?$AAW@ 10001900     hwinit.obj
 0001:00000958       ??_C@_1FI@KPMEKFHG@?$AA?7?$AA?7?$AAW?$AAa?$AAk?$AAe?$AA?5?$AAo?$AAn?$AA?5?$AAD?$AAi?$AAs?$AAc?$AAo?$AAn?$AAn?$AAe?$AAc?$AAt?$AA?5?$AAE?$AAn?$AAa?$AAb?$AAl?$AAe?$AA?5?$AA?$CI?$AAW?$AAK?$AAD@ 10001958     hwinit.obj
 0001:000009b0       ??_C@_1EM@HPIOFCNI@?$AA?7?$AA?7?$AAW?$AAa?$AAk?$AAe?$AA?5?$AAo?$AAn?$AA?5?$AAC?$AAo?$AAn?$AAn?$AAe?$AAc?$AAt?$AA?5?$AAE?$AAn?$AAa?$AAb?$AAl?$AAe?$AA?5?$AA?$CI?$AAW?$AAK?$AAC?$AAN?$AAN?$AAT@ 100019b0     hwinit.obj
 0001:000009fc       ??_C@_1DE@NJCPBMGI@?$AA?7?$AA?7?$AAP?$AAo?$AAr?$AAt?$AA?5?$AAT?$AAe?$AAs?$AAt?$AA?5?$AAC?$AAo?$AAn?$AAt?$AAr?$AAo?$AAl?$AA?3?$AA?5?$AA?$CF?$AAx?$AA?$AN?$AA?6?$AA?$AA@ 100019fc     hwinit.obj
 0001:00000a30       ??_C@_1BG@LAPJBFLO@?$AA?7?$AA?7?$AA?7?$AAG?$AAr?$AAe?$AAe?$AAn?$AA?$AN?$AA?6?$AA?$AA@ 10001a30     hwinit.obj
 0001:00000a48       ??_C@_1BG@IMMCDJCL@?$AA?7?$AA?7?$AA?7?$AAA?$AAm?$AAb?$AAe?$AAr?$AA?$AN?$AA?6?$AA?$AA@ 10001a48     hwinit.obj
 0001:00000a60       ??_C@_1DC@IPGABND@?$AA?7?$AA?7?$AAP?$AAo?$AAr?$AAt?$AA?5?$AAI?$AAn?$AAd?$AAi?$AAc?$AAa?$AAt?$AAo?$AAr?$AA?5?$AAC?$AAo?$AAn?$AAt?$AAr?$AAo?$AAl?$AA?$AA@ 10001a60     hwinit.obj
 0001:00000a94       ??_C@_1BO@FPLCLNEP@?$AA?7?$AA?7?$AAP?$AAo?$AAr?$AAt?$AA?5?$AAO?$AAw?$AAn?$AAe?$AAr?$AA?$AN?$AA?6?$AA?$AA@ 10001a94     hwinit.obj
 0001:00000ab4       ??_C@_1DO@MCLJLJA@?$AA?7?$AA?7?$AA?$DP?$AA?$DP?$AA?$DP?$AA?5?$AAS?$AAh?$AAo?$AAu?$AAl?$AAd?$AA?5?$AAb?$AAe?$AA?5?$AA0?$AA?5?$AAf?$AAo?$AAr?$AA?5?$AAd?$AAe?$AAv?$AAi?$AAc?$AAe?$AA?$AN?$AA?6?$AA?$AA@ 10001ab4     hwinit.obj
 0001:00000af4       ??_C@_1BO@CGJIBKMJ@?$AA?7?$AA?7?$AA?7?$AAU?$AAn?$AAd?$AAe?$AAf?$AAi?$AAn?$AAe?$AAd?$AA?$AN?$AA?6?$AA?$AA@ 10001af4     hwinit.obj
 0001:00000b14       ??_C@_1BK@LEBDPOFP@?$AA?7?$AA?7?$AA?7?$AAK?$AA?9?$AAs?$AAt?$AAa?$AAt?$AAe?$AA?$AN?$AA?6?$AA?$AA@ 10001b14     hwinit.obj
 0001:00000b30       ??_C@_1BK@NBHEMFBJ@?$AA?7?$AA?7?$AA?7?$AAJ?$AA?9?$AAs?$AAt?$AAa?$AAt?$AAe?$AA?$AN?$AA?6?$AA?$AA@ 10001b30     hwinit.obj
 0001:00000b4c       ??_C@_1BC@HGFCDNBO@?$AA?7?$AA?7?$AA?7?$AAS?$AAE?$AA0?$AA?$AN?$AA?6?$AA?$AA@ 10001b4c     hwinit.obj
 0001:00000b60       ??_C@_1CE@HKBMNK@?$AA?7?$AA?7?$AAL?$AAi?$AAn?$AAe?$AA?5?$AAS?$AAt?$AAa?$AAt?$AAu?$AAs?$AA?3?$AA?5?$AA?$CF?$AAx?$AA?$AA@ 10001b60     hwinit.obj
 0001:00000b84       ??_C@_1CK@KAKGINHH@?$AA?7?$AA?7?$AAH?$AAi?$AAg?$AAh?$AA?9?$AAS?$AAp?$AAe?$AAe?$AAd?$AA?5?$AAP?$AAo?$AAr?$AAt?$AA?5?$AA?$AN?$AA?6?$AA?$AA@ 10001b84     hwinit.obj
 0001:00000bb0       ??_C@_1BO@GDNLNMNM@?$AA?7?$AA?7?$AAP?$AAo?$AAr?$AAt?$AA?5?$AAR?$AAe?$AAs?$AAe?$AAt?$AA?$AN?$AA?6?$AA?$AA@ 10001bb0     hwinit.obj
 0001:00000bd0       ??_C@_1BI@BCOEFLFO@?$AA?7?$AA?7?$AAS?$AAu?$AAs?$AAp?$AAe?$AAn?$AAd?$AA?$AN?$AA?6?$AA?$AA@ 10001bd0     hwinit.obj
 0001:00000be8       ??_C@_1CM@LOGLIGHF@?$AA?7?$AA?7?$AAF?$AAo?$AAr?$AAc?$AAe?$AA?5?$AAP?$AAo?$AAr?$AAt?$AA?5?$AAR?$AAe?$AAs?$AAu?$AAm?$AAe?$AA?$AN?$AA?6?$AA?$AA@ 10001be8     hwinit.obj
 0001:00000c14       ??_C@_1DA@IPBKEGAM@?$AA?7?$AA?7?$AAO?$AAv?$AAe?$AAr?$AA?9?$AAc?$AAu?$AAr?$AAr?$AAe?$AAn?$AAt?$AA?5?$AAC?$AAh?$AAa?$AAn?$AAg?$AAe?$AA?$AN?$AA?6?$AA?$AA@ 10001c14     hwinit.obj
 0001:00000c44       ??_C@_1DA@IOPAFHGK@?$AA?7?$AA?7?$AAO?$AAv?$AAe?$AAr?$AA?9?$AAc?$AAu?$AAr?$AAr?$AAe?$AAn?$AAt?$AA?5?$AAA?$AAc?$AAt?$AAi?$AAv?$AAe?$AA?$AN?$AA?6?$AA?$AA@ 10001c44     hwinit.obj
 0001:00000c74       ??_C@_1DO@IDEEGAC@?$AA?7?$AA?7?$AAP?$AAo?$AAr?$AAt?$AA?5?$AAE?$AAn?$AAa?$AAb?$AAl?$AAe?$AA?1?$AAD?$AAi?$AAs?$AAa?$AAb?$AAl?$AAe?$AA?5?$AAC?$AAh?$AAa?$AAn?$AAg?$AAe?$AA?$AN?$AA?6?$AA?$AA@ 10001c74     hwinit.obj
 0001:00000cb4       ??_C@_1CC@HIBPLHBD@?$AA?7?$AA?7?$AAP?$AAo?$AAr?$AAt?$AA?5?$AAE?$AAn?$AAa?$AAb?$AAl?$AAe?$AAd?$AA?$AN?$AA?6?$AA?$AA@ 10001cb4     hwinit.obj
 0001:00000cd8       ??_C@_1EG@CHIFACHN@?$AA?7?$AA?7?$AAC?$AAo?$AAn?$AAn?$AAe?$AAc?$AAt?$AA?5?$AAS?$AAt?$AAa?$AAt?$AAu?$AAs?$AA?5?$AAC?$AAh?$AAa?$AAn?$AAg?$AAe?$AA?3?$AA?5?$AAC?$AAh?$AAa?$AAn?$AAg?$AAe?$AAd@ 10001cd8     hwinit.obj
 0001:00000d20       ??_C@_1EK@CIGPBIFB@?$AA?7?$AA?7?$AAC?$AAu?$AAr?$AAr?$AAe?$AAn?$AAt?$AA?5?$AAC?$AAo?$AAn?$AAn?$AAe?$AAc?$AAt?$AA?5?$AAS?$AAt?$AAa?$AAt?$AAu?$AAs?$AA?3?$AA?5?$AAA?$AAt?$AAt?$AAa?$AAc?$AAh@ 10001d20     hwinit.obj
 0001:00000d6c       ??_C@_1CG@FJJIMMGB@?$AAC?$AAo?$AAn?$AAf?$AAi?$AAg?$AA?5?$AAX?$AAV?$AAC?$AA?5?$AAa?$AAs?$AA?5?$AA?$CF?$AAs?$AA?$AN?$AA?6?$AA?$AA@ 10001d6c     hwinit.obj
 0001:00000d94       ??_C@_17CBGHINCI@?$AAD?$AAe?$AAv?$AA?$AA@ 10001d94     hwinit.obj
 0001:00000d9c       ??_C@_19PBDICKGO@?$AAH?$AAo?$AAs?$AAt?$AA?$AA@ 10001d9c     hwinit.obj
 0001:00000da8       ??_C@_1CC@DEBCAHKH@?$AA?9?$AAC?$AAo?$AAn?$AAf?$AAi?$AAg?$AAO?$AAT?$AAG?$AAH?$AAo?$AAs?$AAt?$AA?$AN?$AA?6?$AA?$AA@ 10001da8     hwinit.obj
 0001:00000dcc       ??_C@_1DM@NCNLGOJP@?$AAH?$AAo?$AAs?$AAt?$AA?5?$AAd?$AAo?$AAe?$AAs?$AA?5?$AAn?$AAo?$AAt?$AA?5?$AAc?$AAo?$AAn?$AAt?$AAr?$AAo?$AAl?$AA?5?$AAp?$AAo?$AAw?$AAe?$AAr?$AA?$AN?$AA?6?$AA?$AA@ 10001dcc     hwinit.obj
 0001:00000e08       ??_C@_1CC@OPBPOBBD@?$AA?$CL?$AAC?$AAo?$AAn?$AAf?$AAi?$AAg?$AAO?$AAT?$AAG?$AAH?$AAo?$AAs?$AAt?$AA?$AN?$AA?6?$AA?$AA@ 10001e08     hwinit.obj
 0001:00000e2c       ??_C@_1DE@FBNMCEFD@?$AAC?$AAo?$AAn?$AAf?$AAi?$AAg?$AAO?$AAT?$AAG?$AAC?$AAl?$AAi?$AAe?$AAn?$AAt?$AA?5?$AAi?$AAs?$AA?5?$AAd?$AAo?$AAn?$AAe?$AA?$AN?$AA?6?$AA?$AA@ 10001e2c     hwinit.obj
 0001:00000e60       ??_C@_1CI@CHEBDPJ@?$AA?9?$AAR?$AAe?$AAg?$AAi?$AAs?$AAt?$AAe?$AAr?$AAC?$AAa?$AAl?$AAl?$AAb?$AAa?$AAc?$AAk?$AA?$AN?$AA?6?$AA?$AA@ 10001e60     hwinit.obj
 0001:00000e88       ??_C@_1DG@FBPLAND@?$AAR?$AAe?$AAg?$AAi?$AAs?$AAt?$AAe?$AAr?$AAC?$AAa?$AAl?$AAl?$AAb?$AAa?$AAc?$AAk?$AA?5?$AAf?$AAo?$AAr?$AA?5?$AAX?$AAV?$AAC?$AA?$AN?$AA?6?$AA?$AA@ 10001e88     hwinit.obj
 0001:00000ec0       ??_C@_1CI@FHANHCOJ@?$AA?$CL?$AAR?$AAe?$AAg?$AAi?$AAs?$AAt?$AAe?$AAr?$AAC?$AAa?$AAl?$AAl?$AAb?$AAa?$AAc?$AAk?$AA?$AN?$AA?6?$AA?$AA@ 10001ec0     hwinit.obj
 0001:00000ee8       ??_C@_1FA@CBCGBFHF@?$AAB?$AAS?$AAP?$AAU?$AAs?$AAb?$AAX?$AAv?$AAr?$AAS?$AAe?$AAt?$AAP?$AAh?$AAy?$AAP?$AAo?$AAw?$AAe?$AAr?$AAM?$AAo?$AAd?$AAe?$AA?5?$AAb?$AAR?$AAe?$AAs?$AAu?$AAm?$AAe@ 10001ee8     hwinit.obj
 0001:00000fc8       ??_C@_1GM@KKEMFHME@?$AA?9?$AAP?$AAo?$AAr?$AAt?$AA?$CI?$AA?$CF?$AAd?$AA?$CJ?$AA?3?$AAB?$AAS?$AAP?$AAU?$AAS?$AAB?$AAC?$AAl?$AAo?$AAc?$AAk?$AAC?$AAr?$AAe?$AAa?$AAt?$AAe?$AAF?$AAi?$AAl?$AAe?$AAM@ 10001fc8     i_usbclock.obj
 0001:00001038       ??_C@_1GO@KPNBKEAO@?$AAP?$AAo?$AAr?$AAt?$AA?$CI?$AA?$CF?$AAd?$AA?$CJ?$AA?3?$AAB?$AAS?$AAP?$AAU?$AAS?$AAB?$AAC?$AAl?$AAo?$AAc?$AAk?$AAC?$AAr?$AAe?$AAa?$AAt?$AAe?$AAF?$AAi?$AAl?$AAe?$AAM?$AAa@ 10002038     i_usbclock.obj
 0001:000010a8       ??_C@_1FE@GNDFGBM@?$AAP?$AAo?$AAr?$AAt?$AA?$CI?$AA?$CF?$AAd?$AA?$CJ?$AA?5?$AAO?$AAp?$AAe?$AAn?$AA?5?$AAe?$AAx?$AAi?$AAs?$AAt?$AAi?$AAn?$AAg?$AA?5?$AAU?$AAS?$AAB?$AA_?$AAC?$AAL?$AAO?$AAC?$AAK@ 100020a8     i_usbclock.obj
 0001:00001100       ??_C@_1FI@ECFJDMMH@?$AAP?$AAo?$AAr?$AAt?$AA?$CI?$AA?$CF?$AAd?$AA?$CJ?$AA?3?$AAF?$AAi?$AAr?$AAs?$AAt?$AA?5?$AAt?$AAo?$AA?5?$AAc?$AAr?$AAe?$AAa?$AAt?$AAe?$AA?5?$AAU?$AAS?$AAB?$AA_?$AAC?$AAL?$AAO@ 10002100     i_usbclock.obj
 0001:00001158       ??_C@_1FC@NEMMIEIK@?$AAF?$AAa?$AAi?$AAl?$AAu?$AAr?$AAe?$AA?5?$AAt?$AAo?$AA?5?$AAC?$AAr?$AAe?$AAa?$AAt?$AAe?$AA?5?$AAF?$AAi?$AAl?$AAe?$AA?5?$AAM?$AAa?$AAp?$AAp?$AAi?$AAn?$AAg?$AA?5?$AAf@ 10002158     i_usbclock.obj
 0001:000011ac       ??_C@_1CC@BJPGGDNC@?$AAU?$AAS?$AAB?$AA_?$AAC?$AAL?$AAO?$AAC?$AAK?$AA_?$AAG?$AAA?$AAT?$AAI?$AAN?$AAG?$AA?$AA@ 100021ac     i_usbclock.obj
 0001:000011d0       ??_C@_1EG@CGIBPELK@?$AAP?$AAo?$AAr?$AAt?$AA?$CI?$AA?$CF?$AAd?$AA?$CJ?$AA?3?$AAB?$AAS?$AAP?$AAU?$AAS?$AAB?$AAC?$AAr?$AAe?$AAa?$AAt?$AAe?$AAF?$AAi?$AAl?$AAe?$AAM?$AAa?$AAp?$AAp?$AAi?$AAn?$AAg@ 100021d0     i_usbclock.obj
 0001:00001218       ??_C@_1IC@FDNBOOON@?$AAP?$AAo?$AAr?$AAt?$AA?$CI?$AA?$CF?$AAd?$AA?$CJ?$AA?5?$AA?9?$AA?5?$AAU?$AAS?$AAB?$AAC?$AAl?$AAo?$AAc?$AAk?$AAC?$AAa?$AAn?$AAC?$AAl?$AAo?$AAc?$AAk?$AAG?$AAa?$AAt?$AAi?$AAn@ 10002218     i_usbclock.obj
 0001:0000129c       ??_C@_1DA@CLIJDNJA@?$AAU?$AAS?$AAB?$AAC?$AAl?$AAo?$AAc?$AAk?$AA?5?$AA?$CF?$AAs?$AA?5?$AAr?$AAe?$AAt?$AAu?$AAr?$AAn?$AA?5?$AA?$CF?$AAd?$AA?$AN?$AA?6?$AA?$AA@ 1000229c     i_usbclock.obj
 0001:000012cc       ??_C@_1M@HCOOECOK@?$AAF?$AAA?$AAL?$AAS?$AAE?$AA?$AA@ 100022cc     i_usbclock.obj
 0001:000012d8       ??_C@_19ELAAHEEL@?$AAT?$AAR?$AAU?$AAE?$AA?$AA@ 100022d8     i_usbclock.obj
 0001:000012e8       ??_C@_1FM@HIIFJIHO@?$AAD?$AAi?$AAs?$AAa?$AAb?$AAl?$AAe?$AA?5?$AAF?$AAa?$AAi?$AAl?$AA?0?$AA?5?$AAN?$AAe?$AAe?$AAd?$AA?5?$AAt?$AAo?$AA?5?$AAc?$AAh?$AAe?$AAc?$AAk?$AA?0?$AA?5?$AAc?$AAu?$AAr@ 100022e8     i_usbclock.obj
 0001:00001348       ??_C@_1FK@HJNHKCPL@?$AAE?$AAn?$AAa?$AAb?$AAl?$AAe?$AA?5?$AAF?$AAa?$AAi?$AAl?$AA?0?$AA?5?$AAN?$AAe?$AAe?$AAd?$AA?5?$AAt?$AAo?$AA?5?$AAc?$AAh?$AAe?$AAc?$AAk?$AA?0?$AA?5?$AAc?$AAu?$AAr?$AAr@ 10002348     i_usbclock.obj
 0001:000013a8       ??_C@_1FI@MBIBGPGK@?$AAU?$AAS?$AAB?$AAC?$AAl?$AAo?$AAc?$AAk?$AAS?$AAe?$AAt?$AA?3?$AA?5?$AAD?$AAD?$AAK?$AAC?$AAl?$AAo?$AAc?$AAk?$AAS?$AAe?$AAt?$AAG?$AAa?$AAt?$AAi?$AAn?$AAg?$AAM?$AAo@ 100023a8     i_usbclock.obj
 0001:00001400       ??_C@_1FC@PCOPMCOB@?$AAU?$AAS?$AAB?$AAC?$AAl?$AAo?$AAc?$AAk?$AAS?$AAe?$AAt?$AA?3?$AA?5?$AAD?$AAD?$AAK?$AAC?$AAl?$AAo?$AAc?$AAk?$AAC?$AAo?$AAn?$AAf?$AAi?$AAg?$AAB?$AAa?$AAu?$AAd?$AA?5@ 10002400     i_usbclock.obj
 0001:000014e8       ??_C@_1EK@IBIELIGM@?$AAC?$AAa?$AAn?$AAn?$AAo?$AAt?$AA?5?$AAo?$AAb?$AAt?$AAa?$AAi?$AAn?$AA?5?$AAt?$AAh?$AAe?$AA?5?$AAs?$AAi?$AAl?$AAi?$AAc?$AAo?$AAn?$AA?5?$AAv?$AAe?$AAr?$AAs?$AAi?$AAo@ 100024e8     i_usbutils.obj
 0001:00001534       ??_C@_1CI@OHCJFJPM@?$AAE?$AAR?$AAR?$AAO?$AAR?$AA?3?$AA?5?$AA?$CF?$AAs?$AA?5?$AAl?$AAi?$AAn?$AAe?$AA?5?$AA?$CF?$AAd?$AA?3?$AA?5?$AA?$AA@ 10002534     i_usbutils.obj
 0001:0000155c       ??_C@_1DE@DKKKIJG@?$AA?4?$AA?2?$AA?4?$AA?4?$AA?2?$AAU?$AAS?$AAB?$AAC?$AAo?$AAm?$AAm?$AAo?$AAn?$AA?2?$AAU?$AAs?$AAb?$AAU?$AAt?$AAi?$AAl?$AAs?$AA?4?$AAc?$AA?$AA@ 1000255c     i_usbutils.obj
 0001:00001590       ??_C@_1BC@GDFGLIEL@?$AAO?$AAT?$AAG?$AAG?$AAr?$AAo?$AAu?$AAp?$AA?$AA@ 10002590     usb_xvc_mx25_topaz_v1:i_xvc.obj
 0001:000015a4       ??_C@_1BG@HHFAGDDC@?$AAO?$AAT?$AAG?$AAS?$AAu?$AAp?$AAp?$AAo?$AAr?$AAt?$AA?$AA@ 100025a4     usb_xvc_mx25_topaz_v1:i_xvc.obj
 0001:000015bc       ??_C@_17DJGGJCGD@?$AAI?$AAr?$AAq?$AA?$AA@ 100025bc     usb_xvc_mx25_topaz_v1:i_xvc.obj
 0001:000015c4       ??_C@_1O@LBBNFMDB@?$AAM?$AAe?$AAm?$AAL?$AAe?$AAn?$AA?$AA@ 100025c4     usb_xvc_mx25_topaz_v1:i_xvc.obj
 0001:000015d4       ??_C@_1BA@INLDIDEN@?$AAM?$AAe?$AAm?$AAB?$AAa?$AAs?$AAe?$AA?$AA@ 100025d4     usb_xvc_mx25_topaz_v1:i_xvc.obj
 0001:000016f0       ??_C@_1EG@JKFFHBLF@?$AAX?$AAV?$AAC?$AA_?$AAD?$AAl?$AAl?$AAE?$AAn?$AAt?$AAr?$AAy?$AA?3?$AA?5?$AAD?$AAL?$AAL?$AA_?$AAP?$AAR?$AAO?$AAC?$AAE?$AAS?$AAS?$AA_?$AAD?$AAE?$AAT?$AAA?$AAC?$AAH@ 100026f0     usb_xvc_mx25_topaz_v1:i_xvc.obj
 0001:00001738       ??_C@_1EG@DGOALPFN@?$AAX?$AAV?$AAC?$AA_?$AAD?$AAl?$AAl?$AAE?$AAn?$AAt?$AAr?$AAy?$AA?3?$AA?5?$AAD?$AAL?$AAL?$AA_?$AAP?$AAR?$AAO?$AAC?$AAE?$AAS?$AAS?$AA_?$AAA?$AAT?$AAT?$AAA?$AAC?$AAH@ 10002738     usb_xvc_mx25_topaz_v1:i_xvc.obj
 0001:00001780       ??_C@_1BO@CMEEGJFP@?$AAX?$AAV?$AAC?$AA_?$AAI?$AAS?$AAT?$AAM?$AAa?$AAi?$AAn?$AA?9?$AA?$AN?$AA?6?$AA?$AA@ 10002780     usb_xvc_mx25_topaz_v1:i_xvc.obj
 0001:000017a0       ??_C@_1HI@MMCNNPDD@?$AAX?$AAV?$AAC?$AA_?$AAI?$AAn?$AAi?$AAt?$AA?3?$AA?5?$AAI?$AAn?$AAt?$AAe?$AAr?$AAr?$AAu?$AAp?$AAt?$AA?5?$AAi?$AAn?$AAi?$AAt?$AAi?$AAa?$AAl?$AAi?$AAz?$AAa?$AAt?$AAi@ 100027a0     usb_xvc_mx25_topaz_v1:i_xvc.obj
 0001:00001818       ??_C@_1CO@MEKJEMED@?$AAX?$AAV?$AAR?$AA?5?$AAI?$AAn?$AA?5?$AAc?$AAo?$AAn?$AAt?$AAr?$AAo?$AAl?$AA?5?$AAa?$AAg?$AAa?$AAi?$AAn?$AA?$AN?$AA?6?$AA?$AA@ 10002818     usb_xvc_mx25_topaz_v1:i_xvc.obj
 0001:00001848       ??_C@_1DK@NFDFBJIJ@?$AAA?$AA?9?$AAd?$AAe?$AAv?$AAi?$AAc?$AAe?$AA?5?$AAh?$AAo?$AAs?$AAt?$AA?5?$AAf?$AAr?$AAo?$AAm?$AA?5?$AAp?$AAo?$AAl?$AAl?$AAi?$AAn?$AAg?$AA?$AN?$AA?6?$AA?$AA@ 10002848     usb_xvc_mx25_topaz_v1:i_xvc.obj
 0001:00001884       ??_C@_1CA@PHGJMMMI@?$AAA?$AA?9?$AAD?$AAe?$AAv?$AAi?$AAc?$AAe?$AA?5?$AAh?$AAo?$AAs?$AAt?$AA?$AN?$AA?6?$AA?$AA@ 10002884     usb_xvc_mx25_topaz_v1:i_xvc.obj
 0001:000018a4       ??_C@_1CE@HPEECKPB@?$AAB?$AA?9?$AAD?$AAe?$AAv?$AAi?$AAc?$AAe?$AA?5?$AAc?$AAl?$AAi?$AAe?$AAn?$AAt?$AA?$AN?$AA?6?$AA?$AA@ 100028a4     usb_xvc_mx25_topaz_v1:i_xvc.obj
 0001:000018c8       ??_C@_1CA@LKDPOEKK@?$AAX?$AAV?$AAC?$AA?5?$AA?9?$AA?5?$AAS?$AAU?$AAS?$AAP?$AAE?$AAN?$AAD?$AA?$AN?$AA?6?$AA?$AA@ 100028c8     usb_xvc_mx25_topaz_v1:i_xvc.obj
 0001:000018e8       ??_C@_1EM@BLHGFICD@?$AAX?$AAC?$AAV?$AAR?$AA?3?$AA?5?$AAC?$AAr?$AAe?$AAa?$AAt?$AAe?$AA?5?$AAE?$AAv?$AAe?$AAn?$AAt?$AA?5?$AAF?$AAa?$AAi?$AAl?$AAe?$AAd?$AA?5?$AAf?$AAo?$AAr?$AA?5?$AAh?$AAo@ 100028e8     usb_xvc_mx25_topaz_v1:i_xvc.obj
 0001:00001938       ??_C@_1EC@IEOCEAJI@?$AAX?$AAC?$AAV?$AAR?$AA?3?$AA?5?$AAC?$AAr?$AAe?$AAa?$AAt?$AAe?$AAd?$AA?5?$AAa?$AA?5?$AAn?$AAe?$AAw?$AA?5?$AAH?$AAo?$AAs?$AAt?$AA?5?$AAE?$AAv?$AAe?$AAn?$AAt?$AA?$AN?$AA?6@ 10002938     usb_xvc_mx25_topaz_v1:i_xvc.obj
 0001:00001980       ??_C@_1EM@NBGKPPCG@?$AAX?$AAC?$AAV?$AAR?$AA?3?$AA?5?$AAO?$AAp?$AAe?$AAn?$AAe?$AAd?$AA?5?$AAa?$AAn?$AA?5?$AAe?$AAx?$AAi?$AAs?$AAt?$AAi?$AAn?$AAg?$AA?5?$AAH?$AAo?$AAs?$AAt?$AA?5?$AAE?$AAv@ 10002980     usb_xvc_mx25_topaz_v1:i_xvc.obj
 0001:000019cc       ??_C@_1BA@MLDLNLBG@?$AAU?$AAS?$AAB?$AAH?$AAo?$AAs?$AAt?$AA?$AA@ 100029cc     usb_xvc_mx25_topaz_v1:i_xvc.obj
 0001:000019e0       ??_C@_1EM@MPCOCLEK@?$AAX?$AAC?$AAV?$AAR?$AA?3?$AA?5?$AAC?$AAr?$AAe?$AAa?$AAt?$AAe?$AA?5?$AAE?$AAv?$AAe?$AAn?$AAt?$AA?5?$AAF?$AAa?$AAi?$AAl?$AAe?$AAd?$AA?5?$AAf?$AAo?$AAr?$AA?5?$AAX?$AAC@ 100029e0     usb_xvc_mx25_topaz_v1:i_xvc.obj
 0001:00001a30       ??_C@_1EC@DGKEOPKG@?$AAX?$AAC?$AAV?$AAR?$AA?3?$AA?5?$AAC?$AAr?$AAe?$AAa?$AAt?$AAe?$AAd?$AA?5?$AAa?$AA?5?$AAn?$AAe?$AAw?$AA?5?$AAX?$AAC?$AAV?$AAR?$AA?5?$AAE?$AAv?$AAe?$AAn?$AAt?$AA?$AN?$AA?6@ 10002a30     usb_xvc_mx25_topaz_v1:i_xvc.obj
 0001:00001a78       ??_C@_1EM@GDCMFABI@?$AAX?$AAC?$AAV?$AAR?$AA?3?$AA?5?$AAO?$AAp?$AAe?$AAn?$AAe?$AAd?$AA?5?$AAa?$AAn?$AA?5?$AAe?$AAx?$AAi?$AAs?$AAt?$AAi?$AAn?$AAg?$AA?5?$AAX?$AAC?$AAV?$AAR?$AA?5?$AAE?$AAv@ 10002a78     usb_xvc_mx25_topaz_v1:i_xvc.obj
 0001:00001ac4       ??_C@_1BA@JAHEEJIA@?$AAU?$AAS?$AAB?$AAX?$AAC?$AAV?$AAR?$AA?$AA@ 10002ac4     usb_xvc_mx25_topaz_v1:i_xvc.obj
 0001:00001ad8       ??_C@_1EM@NILEDOPM@?$AAX?$AAC?$AAV?$AAR?$AA?3?$AA?5?$AAC?$AAr?$AAe?$AAa?$AAt?$AAe?$AA?5?$AAE?$AAv?$AAe?$AAn?$AAt?$AA?5?$AAF?$AAa?$AAi?$AAl?$AAe?$AAd?$AA?5?$AAf?$AAo?$AAr?$AA?5?$AAf?$AAu@ 10002ad8     usb_xvc_mx25_topaz_v1:i_xvc.obj
 0001:00001b28       ??_C@_1EC@MAPHKJCO@?$AAX?$AAC?$AAV?$AAR?$AA?3?$AA?5?$AAC?$AAr?$AAe?$AAa?$AAt?$AAe?$AAd?$AA?5?$AAa?$AA?5?$AAn?$AAe?$AAw?$AA?5?$AAF?$AAu?$AAn?$AAc?$AA?5?$AAE?$AAv?$AAe?$AAn?$AAt?$AA?$AN?$AA?6@ 10002b28     usb_xvc_mx25_topaz_v1:i_xvc.obj
 0001:00001b70       ??_C@_1EM@JFHPBGJA@?$AAX?$AAC?$AAV?$AAR?$AA?3?$AA?5?$AAO?$AAp?$AAe?$AAn?$AAe?$AAd?$AA?5?$AAa?$AAn?$AA?5?$AAe?$AAx?$AAi?$AAs?$AAt?$AAi?$AAn?$AAg?$AA?5?$AAF?$AAu?$AAn?$AAc?$AA?5?$AAE?$AAv@ 10002b70     usb_xvc_mx25_topaz_v1:i_xvc.obj
 0001:00001bbc       ??_C@_1BA@EKAPLICF@?$AAU?$AAS?$AAB?$AAF?$AAu?$AAn?$AAc?$AA?$AA@ 10002bbc     usb_xvc_mx25_topaz_v1:i_xvc.obj
 0001:00001bcc       ??_C@_1BO@OKCLGANI@?$AAX?$AAV?$AAC?$AA_?$AAI?$AAS?$AAT?$AAM?$AAa?$AAi?$AAn?$AA?$CL?$AA?$AN?$AA?6?$AA?$AA@ 10002bcc     usb_xvc_mx25_topaz_v1:i_xvc.obj
 0001:00001bf0       ??_C@_1FO@DFNLJIPA@?$AAU?$AAS?$AAB?$AAC?$AAo?$AAn?$AAt?$AAr?$AAo?$AAl?$AAl?$AAe?$AAr?$AAR?$AAu?$AAn?$AA?$CI?$AA?$CF?$AAd?$AA?$CJ?$AA?3?$AA?5?$AAf?$AAa?$AAi?$AAl?$AAe?$AAd?$AA?5?$AAt?$AAo?$AA?5@ 10002bf0     usb_xvc_mx25_topaz_v1:i_xvc.obj
 0001:00001c50       ??_C@_1HI@FMJPDAIJ@?$AAU?$AAS?$AAB?$AAC?$AAo?$AAn?$AAt?$AAr?$AAo?$AAl?$AAl?$AAe?$AAr?$AAR?$AAu?$AAn?$AA?$CI?$AA1?$AA?$CJ?$AA?3?$AA?5?$AAE?$AAR?$AAR?$AAO?$AAR?$AA?5?$AA?$CD?$AA?$CD?$AA?$CD?$AA?$CD?$AA?$CD@ 10002c50     usb_xvc_mx25_topaz_v1:i_xvc.obj
 0001:00001cc8       ??_C@_1EM@BBPKMFPI@?$AAS?$AAt?$AAo?$AAp?$AA?5?$AAU?$AAS?$AAB?$AA?5?$AAc?$AAo?$AAn?$AAt?$AAr?$AAo?$AAl?$AAl?$AAe?$AAr?$AA?5?$AA?$CI?$AAR?$AAS?$AA?$DN?$AA?$CF?$AAd?$AA?5?$AA?9?$AA?$DO?$AA?5?$AAR?$AAS@ 10002cc8     usb_xvc_mx25_topaz_v1:i_xvc.obj
 0001:00001d18       ??_C@_1EO@GGMICPAJ@?$AAS?$AAt?$AAa?$AAr?$AAt?$AA?5?$AAU?$AAS?$AAB?$AA?5?$AAc?$AAo?$AAn?$AAt?$AAr?$AAo?$AAl?$AAl?$AAe?$AAr?$AA?5?$AA?$CI?$AAR?$AAS?$AA?$DN?$AA?$CF?$AAd?$AA?5?$AA?9?$AA?$DO?$AA?5?$AAR@ 10002d18     usb_xvc_mx25_topaz_v1:i_xvc.obj
 0001:00001d68       ??_C@_1HG@CNLFGGFF@?$AAU?$AAS?$AAB?$AAC?$AAo?$AAn?$AAt?$AAr?$AAo?$AAl?$AAl?$AAe?$AAr?$AAR?$AAe?$AAs?$AAe?$AAt?$AA?3?$AA?5?$AA?$CD?$AA?$CD?$AA?$CD?$AA?$CD?$AA?$CD?$AA?$CD?$AA?$CD?$AA?$CD?$AA?$CD?$AA?5?$AAF?$AAa@ 10002d68     usb_xvc_mx25_topaz_v1:i_xvc.obj
 0001:00001de0       ??_C@_1GI@KIMADIJB@?$AAU?$AAS?$AAB?$AAC?$AAo?$AAn?$AAt?$AAr?$AAo?$AAl?$AAl?$AAe?$AAr?$AAR?$AAe?$AAs?$AAe?$AAt?$AA?3?$AA?5?$AA?$CD?$AA?$CD?$AA?$CD?$AA?$CD?$AA?$CD?$AA?$CD?$AA?$CD?$AA?$CD?$AA?$CD?$AA?$CD?$AA?$CD?$AA?5@ 10002de0     usb_xvc_mx25_topaz_v1:i_xvc.obj
 0001:00001e48       ??_C@_1GM@PONDOELC@?$AAX?$AAV?$AAC?$AA_?$AAI?$AAn?$AAi?$AAt?$AA?3?$AA?5?$AAF?$AAa?$AAi?$AAl?$AAe?$AAd?$AA?5?$AAt?$AAo?$AA?5?$AAc?$AAr?$AAe?$AAa?$AAt?$AAe?$AA?5?$AAI?$AAn?$AAt?$AAe?$AAr@ 10002e48     usb_xvc_mx25_topaz_v1:i_xvc.obj
 0001:00001eb8       ??_C@_1EE@IMEGGAEC@?$AAX?$AAV?$AAC?$AA_?$AAI?$AAn?$AAi?$AAt?$AA?3?$AA?5?$AAI?$AAn?$AAt?$AAe?$AAr?$AAr?$AAu?$AAp?$AAt?$AA?5?$AAi?$AAn?$AAi?$AAt?$AAi?$AAa?$AAl?$AAi?$AAz?$AAe?$AAd?$AA?$AN@ 10002eb8     usb_xvc_mx25_topaz_v1:i_xvc.obj
 0001:00001efc       ??_C@_1DO@BBDIIJGI@?$AAX?$AAV?$AAC?$AA_?$AAI?$AAn?$AAi?$AAt?$AA?3?$AA?5?$AAC?$AAr?$AAe?$AAa?$AAt?$AAe?$AAE?$AAv?$AAe?$AAn?$AAt?$AA?5?$AAf?$AAa?$AAi?$AAl?$AAe?$AAd?$AA?$AN?$AA?6?$AA?$AA@ 10002efc     usb_xvc_mx25_topaz_v1:i_xvc.obj
 0001:00001f40       ??_C@_1GO@JPJGFDDJ@?$AAE?$AAR?$AAR?$AAO?$AAR?$AA?3?$AA?5?$AAX?$AAV?$AAC?$AA_?$AAI?$AAn?$AAi?$AAt?$AA?3?$AA?5?$AAC?$AAo?$AAn?$AAt?$AAr?$AAo?$AAl?$AAl?$AAe?$AAr?$AA?5?$AAr?$AAe?$AAg?$AAi@ 10002f40     usb_xvc_mx25_topaz_v1:i_xvc.obj
 0001:00001fb0       ??_C@_1FA@KANLLNPK@?$AAO?$AAT?$AAG?$AA?5?$AAN?$AAo?$AAt?$AA?5?$AAs?$AAu?$AAp?$AAp?$AAo?$AAr?$AAt?$AA?5?$AAa?$AAn?$AAd?$AA?5?$AAu?$AAn?$AAl?$AAo?$AAa?$AAd?$AA?5?$AAt?$AAh?$AAe?$AA?5?$AAd@ 10002fb0     usb_xvc_mx25_topaz_v1:i_xvc.obj
 0001:00002000       ??_C@_1GG@GDOKGIEN@?$AAE?$AAR?$AAR?$AAO?$AAR?$AA?3?$AA?5?$AAX?$AAV?$AAC?$AA_?$AAI?$AAn?$AAi?$AAt?$AA?3?$AA?5?$AAF?$AAa?$AAi?$AAl?$AAe?$AAd?$AA?5?$AAr?$AAe?$AAa?$AAd?$AA?5?$AAr?$AAe?$AAg@ 10003000     usb_xvc_mx25_topaz_v1:i_xvc.obj
 0001:00002068       ??_C@_1EG@NGCHCOHA@?$AAX?$AAV?$AAC?$AA_?$AAI?$AAn?$AAi?$AAt?$AA?3?$AA?5?$AAC?$AAa?$AAn?$AAn?$AAo?$AAt?$AA?5?$AAa?$AAl?$AAl?$AAo?$AAc?$AAa?$AAt?$AAe?$AA?5?$AAm?$AAe?$AAm?$AAo?$AAr?$AAy@ 10003068     usb_xvc_mx25_topaz_v1:i_xvc.obj
 0001:000020b0       ??_C@_1GC@KCPKFPFA@?$AAU?$AAS?$AAB?$AA?5?$AA?5?$AAX?$AAV?$AAC?$AA?5?$AAl?$AAo?$AAa?$AAd?$AA?5?$AAf?$AAa?$AAi?$AAl?$AAu?$AAr?$AAe?$AA?5?$AAb?$AAe?$AAc?$AAa?$AAu?$AAs?$AAe?$AA?5?$AAU?$AAs@ 100030b0     usb_xvc_mx25_topaz_v1:i_xvc.obj
 0001:00002114       ??_C@_1BM@MFPICHP@?$AA?9?$AAX?$AAV?$AAC?$AA_?$AAD?$AAe?$AAi?$AAn?$AAi?$AAt?$AA?$AN?$AA?6?$AA?$AA@ 10003114     usb_xvc_mx25_topaz_v1:i_xvc.obj
 0001:00002130       ??_C@_1EA@GLHOIBMK@?$AA?$CL?$AAX?$AAV?$AAC?$AA_?$AAD?$AAe?$AAi?$AAn?$AAi?$AAt?$AA?3?$AA?5?$AAd?$AAw?$AAC?$AAo?$AAn?$AAt?$AAe?$AAx?$AAt?$AA?5?$AA?$DN?$AA?5?$AA0?$AAx?$AA?$CF?$AAx?$AA?$AN?$AA?6?$AA?$AA@ 10003130     usb_xvc_mx25_topaz_v1:i_xvc.obj
 0001:00002170       ??_C@_1BI@BHHCJLKL@?$AA?9?$AAX?$AAV?$AAC?$AA_?$AAO?$AAp?$AAe?$AAn?$AA?$AN?$AA?6?$AA?$AA@ 10003170     usb_xvc_mx25_topaz_v1:i_xvc.obj
 0001:00002188       ??_C@_1IA@LDMEPOAF@?$AA?$CL?$AAX?$AAV?$AAC?$AA_?$AAO?$AAp?$AAe?$AAn?$AA?3?$AA?5?$AAd?$AAw?$AAD?$AAa?$AAt?$AAa?$AA?5?$AA?$DN?$AA?5?$AA0?$AAx?$AA?$CF?$AAx?$AA?0?$AA?5?$AAd?$AAw?$AAA?$AAc?$AAc?$AAe@ 10003188     usb_xvc_mx25_topaz_v1:i_xvc.obj
 0001:00002208       ??_C@_1DI@OBFJAKL@?$AA?9?$AAX?$AAV?$AAC?$AA_?$AAC?$AAl?$AAo?$AAs?$AAe?$AA?3?$AA?5?$AAH?$AAa?$AAn?$AAd?$AAl?$AAe?$AA?5?$AA?$DN?$AA?5?$AA0?$AAx?$AA?$CF?$AAx?$AA?$AN?$AA?6?$AA?$AA@ 10003208     usb_xvc_mx25_topaz_v1:i_xvc.obj
 0001:00002240       ??_C@_1DI@EDGLPIFJ@?$AA?$CL?$AAX?$AAV?$AAC?$AA_?$AAC?$AAl?$AAo?$AAs?$AAe?$AA?3?$AA?5?$AAH?$AAa?$AAn?$AAd?$AAl?$AAe?$AA?5?$AA?$DN?$AA?5?$AA0?$AAx?$AA?$CF?$AAx?$AA?$AN?$AA?6?$AA?$AA@ 10003240     usb_xvc_mx25_topaz_v1:i_xvc.obj
 0001:00002278       ??_C@_1HK@NPLFICCO@?$AAX?$AAV?$AAC?$AA_?$AAR?$AAe?$AAa?$AAd?$AA?3?$AA?5?$AAH?$AAa?$AAn?$AAd?$AAl?$AAe?$AA?5?$AA?$DN?$AA?5?$AA0?$AAx?$AA?$CF?$AAx?$AA?0?$AA?5?$AAp?$AAB?$AAu?$AAf?$AAf?$AAe?$AAr@ 10003278     usb_xvc_mx25_topaz_v1:i_xvc.obj
 0001:000022f8       ??_C@_1HM@OIMOELCG@?$AAX?$AAV?$AAC?$AA_?$AAW?$AAr?$AAi?$AAt?$AAe?$AA?3?$AA?5?$AAH?$AAa?$AAn?$AAd?$AAl?$AAe?$AA?5?$AA?$DN?$AA?5?$AA0?$AAx?$AA?$CF?$AAx?$AA?0?$AA?5?$AAp?$AAB?$AAu?$AAf?$AAf?$AAe@ 100032f8     usb_xvc_mx25_topaz_v1:i_xvc.obj
 0001:00002378       ??_C@_1IC@DKACNHPO@?$AAX?$AAV?$AAC?$AA_?$AAS?$AAe?$AAe?$AAk?$AA?3?$AA?5?$AAH?$AAa?$AAn?$AAd?$AAl?$AAe?$AA?5?$AA?$DN?$AA?5?$AA0?$AAx?$AA?$CF?$AAx?$AA?0?$AA?5?$AAl?$AAD?$AAi?$AAs?$AAt?$AAa?$AAn@ 10003378     usb_xvc_mx25_topaz_v1:i_xvc.obj
 0001:000023fc       ??_C@_1CM@LGFBBFDM@?$AAX?$AAV?$AAC?$AA_?$AAI?$AAO?$AAC?$AAT?$AAL?$AA_?$AAP?$AAO?$AAW?$AAE?$AAR?$AA_?$AAS?$AAE?$AAT?$AA?$AN?$AA?6?$AA?$AA@ 100033fc     usb_xvc_mx25_topaz_v1:i_xvc.obj
 0001:00002428       ??_C@_1BK@NIBAJMFP@?$AAN?$AAe?$AAw?$AAD?$AAx?$AA?5?$AA?$DN?$AA?5?$AA?$CF?$AAd?$AA?$AN?$AA?6?$AA?$AA@ 10003428     usb_xvc_mx25_topaz_v1:i_xvc.obj
 0001:00002444       ??_C@_1DA@BHIIDOOI@?$AAX?$AAV?$AAC?$AA_?$AAI?$AAO?$AAC?$AAT?$AAL?$AA_?$AAP?$AAO?$AAW?$AAE?$AAR?$AA_?$AAQ?$AAU?$AAE?$AAR?$AAY?$AA?$AN?$AA?6?$AA?$AA@ 10003444     usb_xvc_mx25_topaz_v1:i_xvc.obj
 0001:00002474       ??_C@_1DO@IDDMIJLF@?$AAX?$AAV?$AAC?$AA_?$AAI?$AAO?$AAC?$AAT?$AAL?$AA_?$AAP?$AAO?$AAW?$AAE?$AAR?$AA_?$AAC?$AAA?$AAP?$AAA?$AAB?$AAI?$AAL?$AAI?$AAT?$AAI?$AAE?$AAS?$AA?$AN?$AA?6?$AA?$AA@ 10003474     usb_xvc_mx25_topaz_v1:i_xvc.obj
 0001:000024b4       ??_C@_1DI@NOJFOLKN@?$AAI?$AAO?$AAC?$AAT?$AAL?$AA_?$AAB?$AAU?$AAS?$AA_?$AAS?$AAE?$AAT?$AA_?$AAP?$AAO?$AAW?$AAE?$AAR?$AA_?$AAS?$AAT?$AAA?$AAT?$AAE?$AA?$AN?$AA?6?$AA?$AA@ 100034b4     usb_xvc_mx25_topaz_v1:i_xvc.obj
 0001:000024ec       ??_C@_1DI@HIENBGG@?$AAI?$AAO?$AAC?$AAT?$AAL?$AA_?$AAB?$AAU?$AAS?$AA_?$AAG?$AAE?$AAT?$AA_?$AAP?$AAO?$AAW?$AAE?$AAR?$AA_?$AAS?$AAT?$AAA?$AAT?$AAE?$AA?$AN?$AA?6?$AA?$AA@ 100034ec     usb_xvc_mx25_topaz_v1:i_xvc.obj
 0001:00002528       ??_C@_1FC@PFHGPBO@?$AA?$CL?$AAX?$AAV?$AAC?$AA_?$AAI?$AAO?$AAC?$AAo?$AAn?$AAt?$AAr?$AAo?$AAl?$AA?3?$AA?5?$AAd?$AAw?$AAI?$AAo?$AAC?$AAo?$AAn?$AAt?$AAr?$AAo?$AAl?$AAC?$AAo?$AAd?$AAe?$AA?5@ 10003528     usb_xvc_mx25_topaz_v1:i_xvc.obj
 0001:0000257c       ??_C@_1BM@MFAIKPFA@?$AA?9?$AAP?$AAo?$AAw?$AAe?$AAr?$AAD?$AAo?$AAw?$AAn?$AA?5?$AA?$AN?$AA?6?$AA?$AA@ 1000357c     usb_xvc_mx25_topaz_v1:i_xvc.obj
 0001:00002598       ??_C@_1BM@MALEKBBO@?$AA?$CL?$AAP?$AAo?$AAw?$AAe?$AAr?$AAD?$AAo?$AAw?$AAn?$AA?5?$AA?$AN?$AA?6?$AA?$AA@ 10003598     usb_xvc_mx25_topaz_v1:i_xvc.obj
 0001:000025d8       BSPGetUSBControllerType    100035d8 f   hwinit.obj
 0001:000025f0       USBOTGVbusControl          100035f0 f   hwinit.obj
 0001:00002604       DumpUSBRegs                10003604 f   hwinit.obj
 0001:00003470       InitializeOTGTransceiver   10004470 f   hwinit.obj
 0001:00004014       GetSysIntr                 10005014 f   hwinit.obj
 0001:0000407c       RegisterCallback           1000507c f   hwinit.obj
 0001:00004268       BSPUsbResetPHY             10005268 f   hwinit.obj
 0001:000042f0       BSPUsbSetPHYEnable         100052f0 f   hwinit.obj
 0001:00004388       USBClockInit               10005388 f   i_usbclock.obj
 0001:000043b4       USBClockGatingLock         100053b4 f   i_usbclock.obj
 0001:00004410       USBClockGatingUnlock       10005410 f   i_usbclock.obj
 0001:0000442c       BSPUSBClockCreateFileMapping 1000542c f   i_usbclock.obj
 0001:00004660       BSPUSBClockDeleteFileMapping 10005660 f   i_usbclock.obj
 0001:000046c4       BSPUSBClockSwitch          100056c4 f   i_usbclock.obj
 0001:000049f8       PowerDownSchemeExist       100059f8 f   i_usbutils.obj
 0001:00004a9c       BSPUsbXvrEnableVBUSIntr    10005a9c f   i_usbutils.obj
 0001:00004b1c       BSPUsbXvrEnableIDIntr      10005b1c f   i_usbutils.obj
 0001:00004b9c       BSPUsbEnableLowPowerIntr   10005b9c f   i_usbutils.obj
 0001:00004bec       BSPUsbSetBusConfig         10005bec f   i_usbutils.obj
 0001:00004c30       BSPUSBInterruptControl     10005c30 f   i_usbutils.obj
 0001:00004c9c       BSPPhyShowDevDiscon        10005c9c f   i_usbutils.obj
 0001:00004cb4       BSPUsbPhyStartUp           10005cb4 f   i_usbutils.obj
 0001:00004cb8       BSPUsbSetCurrentLimitation 10005cb8 f   i_usbutils.obj
 0001:00004ccc       BSPUsbPhyRegDump           10005ccc f   i_usbutils.obj
 0001:00004cd0       BSPUSBSwitchModulePower    10005cd0 f   i_usbutils.obj
 0001:00004ce4       BSPHostDisconDetect        10005ce4 f   i_usbutils.obj
 0001:00004cf8       FslUfnIsUSBKitlEnable      10005cf8 f   usb_xvc_mx25_topaz_v1:i_xvc.obj
 0001:00004d8c       DllEntry                   10005d8c f   usb_xvc_mx25_topaz_v1:i_xvc.obj
 0001:00004f8c       XVC_ISTMain                10005f8c f   usb_xvc_mx25_topaz_v1:i_xvc.obj
 0001:000064e8       XVC_Init                   100074e8 f   usb_xvc_mx25_topaz_v1:i_xvc.obj
 0001:00006bf8       XVC_Deinit                 10007bf8 f   usb_xvc_mx25_topaz_v1:i_xvc.obj
 0001:00006dac       XVC_Open                   10007dac f   usb_xvc_mx25_topaz_v1:i_xvc.obj
 0001:00006ea8       XVC_Close                  10007ea8 f   usb_xvc_mx25_topaz_v1:i_xvc.obj
 0001:00006f9c       XVC_PowerDown              10007f9c f   usb_xvc_mx25_topaz_v1:i_xvc.obj
 0001:00006fa0       XVC_PowerUp                10007fa0 f   usb_xvc_mx25_topaz_v1:i_xvc.obj
 0001:00006fa4       XVC_Read                   10007fa4 f   usb_xvc_mx25_topaz_v1:i_xvc.obj
 0001:00007044       XVC_Write                  10008044 f   usb_xvc_mx25_topaz_v1:i_xvc.obj
 0001:000070e4       XVC_Seek                   100080e4 f   usb_xvc_mx25_topaz_v1:i_xvc.obj
 0001:00007184       XVC_IOControl              10008184 f   usb_xvc_mx25_topaz_v1:i_xvc.obj
 0001:000079c8       GetUSBOTGIRQ               100089c8 f   usb_xvc_mx25_topaz_v1:i_xvc.obj
 0001:000079e0       SetEvent                   100089e0 f i usb_xvc_mx25_topaz_v1:i_xvc.obj
 0001:00007a18       GetCurrentThread           10008a18 f i usb_xvc_mx25_topaz_v1:i_xvc.obj
 0001:00007a30       ResetEvent                 10008a30 f i usb_xvc_mx25_topaz_v1:i_xvc.obj
 0001:00007a68       GetDeviceRegistryParams    10008a68 f   usb_xvc_mx25_topaz_v1:i_registry.obj
 0001:00008514       NKDbgPrintfW               10009514 f   coredll:COREDLL.dll
 0001:00008524       Sleep                      10009524 f   coredll:COREDLL.dll
 0001:00008534       KernelIoControl            10009534 f   coredll:COREDLL.dll
 0001:00008544       InterlockedCompareExchange 10009544 f   coredll:COREDLL.dll
 0001:00008554       GetLastError               10009554 f   coredll:COREDLL.dll
 0001:00008564       MapViewOfFile              10009564 f   coredll:COREDLL.dll
 0001:00008574       CreateFileMappingW         10009574 f   coredll:COREDLL.dll
 0001:00008584       CloseHandle                10009584 f   coredll:COREDLL.dll
 0001:00008594       UnmapViewOfFile            10009594 f   coredll:COREDLL.dll
 0001:000085a4       DisableThreadLibraryCalls  100095a4 f   coredll:COREDLL.dll
 0001:000085b4       CeLogData                  100095b4 f   coredll:COREDLL.dll
 0001:000085c4       StringCchLengthW           100095c4 f   coredll:COREDLL.dll
 0001:000085d4       StringCchVPrintfW          100095d4 f   coredll:COREDLL.dll
 0001:000085e4       ExitThread                 100095e4 f   coredll:COREDLL.dll
 0001:000085f4       InterruptDone              100095f4 f   coredll:COREDLL.dll
 0001:00008604       InterruptInitialize        10009604 f   coredll:COREDLL.dll
 0001:00008614       InterruptDisable           10009614 f   coredll:COREDLL.dll
 0001:00008624       LeaveCriticalSection       10009624 f   coredll:COREDLL.dll
 0001:00008634       EnterCriticalSection       10009634 f   coredll:COREDLL.dll
 0001:00008644       WaitForSingleObject        10009644 f   coredll:COREDLL.dll
 0001:00008654       SetInterruptEvent          10009654 f   coredll:COREDLL.dll
 0001:00008664       CreateEventW               10009664 f   coredll:COREDLL.dll
 0001:00008674       StringCchCatW              10009674 f   coredll:COREDLL.dll
 0001:00008684       StringCchCopyW             10009684 f   coredll:COREDLL.dll
 0001:00008694       EventModify                10009694 f   coredll:COREDLL.dll
 0001:000086a4       LocalFree                  100096a4 f   coredll:COREDLL.dll
 0001:000086b4       CeSetThreadPriority        100096b4 f   coredll:COREDLL.dll
 0001:000086c4       CreateThread               100096c4 f   coredll:COREDLL.dll
 0001:000086d4       InitializeCriticalSection  100096d4 f   coredll:COREDLL.dll
 0001:000086e4       LocalAlloc                 100096e4 f   coredll:COREDLL.dll
 0001:000086f4       SetThreadPriority          100096f4 f   coredll:COREDLL.dll
 0001:00008704       RegCloseKey                10009704 f   coredll:COREDLL.dll
 0001:00008714       RegOpenKeyExW              10009714 f   coredll:COREDLL.dll
 0001:00008724       OpenDeviceKey              10009724 f   coredll:COREDLL.dll
 0001:00008734       RegQueryValueExW           10009734 f   coredll:COREDLL.dll
 0001:00008744       MmUnmapIoSpace             10009744 f   ceddk:CEDDK.dll
 0001:00008754       MmMapIoSpace               10009754 f   ceddk:CEDDK.dll
 0001:00008764       DDKClockSetGatingMode      10009764 f   cspddk:CSPDDK.dll
 0001:00008774       DDKClockGetGatingMode      10009774 f   cspddk:CSPDDK.dll
 0001:00008784       DDKClockConfigBaud         10009784 f   cspddk:CSPDDK.dll
 0001:00008794       _DllEntryCRTStartup        10009794 f   corelib0:pegdentry.obj
 0001:00008804       __security_init_cookie     10009804 f   corelib0:seccinit.obj
 0001:000088cc       __GSHandlerCheck           100098cc f   corelib0:gshandler.obj
 0001:00008914       __GSHandlerCheckCommon     10009914 f   corelib0:gshandler.obj
 0001:000089bc       __security_check_cookie    100099bc f   corelib0:armsecgs.obj
 0001:000089d0       __gsfailure                100099d0 f   corelib0:armsecgs.obj
 0001:00008a14       exit                       10009a14 f   corelib0:cexit.obj
 0001:00008b94       _exit                      10009b94 f   corelib0:cexit.obj
 0001:00008bb8       _cexit                     10009bb8 f   corelib0:cexit.obj
 0001:00008bd4       _c_exit                    10009bd4 f   corelib0:cexit.obj
 0001:00008bf0       GetCurrentProcess          10009bf0 f i corelib0:cexit.obj
 0001:00008c08       _initterm                  10009c08 f   corelib0:crt0dat.obj
 0001:00008c5c       _cinit                     10009c5c f   corelib0:crt0dat.obj
 0001:00008c98       _onexit                    10009c98 f   corelib0:onexit.obj
 0001:00008f9c       atexit                     10009f9c f   corelib0:onexit.obj
 0001:00008ff0       memset                     10009ff0 f   corelib1:COREDLL.dll
 0001:00009000       memcpy                     1000a000 f   corelib1:COREDLL.dll
 0001:00009010       wcslen                     1000a010 f   corelib1:COREDLL.dll
 0001:00009020       wcstoul                    1000a020 f   corelib1:COREDLL.dll
 0001:00009030       __security_gen_cookie2     1000a030 f   corelib1:COREDLL.dll
 0001:00009040       __report_gsfailure         1000a040 f   corelib1:COREDLL.dll
 0001:00009050       free                       1000a050 f   corelib1:COREDLL.dll
 0001:00009060       __C_specific_handler       1000a060 f   corelib1:COREDLL.dll
 0001:00009070       malloc                     1000a070 f   corelib1:COREDLL.dll
 0001:00009080       realloc                    1000a080 f   corelib1:COREDLL.dll
 0001:00009090       _msize                     1000a090 f   corelib1:COREDLL.dll
 0001:000090a0       DeleteCriticalSection      1000a0a0 f   coredll:COREDLL.dll
 0001:000090b0       InterlockedExchange        1000a0b0 f   coredll:COREDLL.dll
 0001:000090c0       TerminateProcess           1000a0c0 f   coredll:COREDLL.dll
 0001:000090ec       __IMPORT_DESCRIPTOR_COREDLL 1000a0ec     coredll:COREDLL.dll
 0001:00009100       __IMPORT_DESCRIPTOR_CEDDK  1000a100     ceddk:CEDDK.dll
 0001:00009114       __IMPORT_DESCRIPTOR_CSPDDK 1000a114     cspddk:CSPDDK.dll
 0001:00009128       __NULL_IMPORT_DESCRIPTOR   1000a128     coredll:COREDLL.dll
 0002:00000000       __imp_MmUnmapIoSpace       1000b000     ceddk:CEDDK.dll
 0002:00000004       __imp_MmMapIoSpace         1000b004     ceddk:CEDDK.dll
 0002:00000008       \177CEDDK_NULL_THUNK_DATA  1000b008     ceddk:CEDDK.dll
 0002:0000000c       __imp_InterlockedCompareExchange 1000b00c     coredll:COREDLL.dll
 0002:00000010       __imp_GetLastError         1000b010     coredll:COREDLL.dll
 0002:00000014       __imp_MapViewOfFile        1000b014     coredll:COREDLL.dll
 0002:00000018       __imp_CreateFileMappingW   1000b018     coredll:COREDLL.dll
 0002:0000001c       __imp_CloseHandle          1000b01c     coredll:COREDLL.dll
 0002:00000020       __imp_UnmapViewOfFile      1000b020     coredll:COREDLL.dll
 0002:00000024       __imp_DisableThreadLibraryCalls 1000b024     coredll:COREDLL.dll
 0002:00000028       __imp_CeLogData            1000b028     coredll:COREDLL.dll
 0002:0000002c       __imp_StringCchLengthW     1000b02c     coredll:COREDLL.dll
 0002:00000030       __imp_StringCchVPrintfW    1000b030     coredll:COREDLL.dll
 0002:00000034       __imp_ExitThread           1000b034     coredll:COREDLL.dll
 0002:00000038       __imp_InterruptDone        1000b038     coredll:COREDLL.dll
 0002:0000003c       __imp_InterruptInitialize  1000b03c     coredll:COREDLL.dll
 0002:00000040       __imp_InterruptDisable     1000b040     coredll:COREDLL.dll
 0002:00000044       __imp_LeaveCriticalSection 1000b044     coredll:COREDLL.dll
 0002:00000048       __imp_EnterCriticalSection 1000b048     coredll:COREDLL.dll
 0002:0000004c       __imp_KernelIoControl      1000b04c     coredll:COREDLL.dll
 0002:00000050       __imp_SetInterruptEvent    1000b050     coredll:COREDLL.dll
 0002:00000054       __imp_CreateEventW         1000b054     coredll:COREDLL.dll
 0002:00000058       __imp_StringCchCatW        1000b058     coredll:COREDLL.dll
 0002:0000005c       __imp_StringCchCopyW       1000b05c     coredll:COREDLL.dll
 0002:00000060       __imp_EventModify          1000b060     coredll:COREDLL.dll
 0002:00000064       __imp_LocalFree            1000b064     coredll:COREDLL.dll
 0002:00000068       __imp_CeSetThreadPriority  1000b068     coredll:COREDLL.dll
 0002:0000006c       __imp_CreateThread         1000b06c     coredll:COREDLL.dll
 0002:00000070       __imp_InitializeCriticalSection 1000b070     coredll:COREDLL.dll
 0002:00000074       __imp_LocalAlloc           1000b074     coredll:COREDLL.dll
 0002:00000078       __imp_SetThreadPriority    1000b078     coredll:COREDLL.dll
 0002:0000007c       __imp_RegCloseKey          1000b07c     coredll:COREDLL.dll
 0002:00000080       __imp_RegOpenKeyExW        1000b080     coredll:COREDLL.dll
 0002:00000084       __imp_OpenDeviceKey        1000b084     coredll:COREDLL.dll
 0002:00000088       __imp_RegQueryValueExW     1000b088     coredll:COREDLL.dll
 0002:0000008c       __imp_Sleep                1000b08c     coredll:COREDLL.dll
 0002:00000090       __imp_WaitForSingleObject  1000b090     coredll:COREDLL.dll
 0002:00000094       __imp_NKDbgPrintfW         1000b094     coredll:COREDLL.dll
 0002:00000098       __imp_InterlockedExchange  1000b098     coredll:COREDLL.dll
 0002:0000009c       __imp_DeleteCriticalSection 1000b09c     coredll:COREDLL.dll
 0002:000000a0       __imp__msize               1000b0a0     corelib1:COREDLL.dll
 0002:000000a4       __imp_realloc              1000b0a4     corelib1:COREDLL.dll
 0002:000000a8       __imp_memset               1000b0a8     corelib1:COREDLL.dll
 0002:000000ac       __imp_memcpy               1000b0ac     corelib1:COREDLL.dll
 0002:000000b0       __imp_wcslen               1000b0b0     corelib1:COREDLL.dll
 0002:000000b4       __imp_wcstoul              1000b0b4     corelib1:COREDLL.dll
 0002:000000b8       __imp___security_gen_cookie2 1000b0b8     corelib1:COREDLL.dll
 0002:000000bc       __imp___report_gsfailure   1000b0bc     corelib1:COREDLL.dll
 0002:000000c0       __imp_free                 1000b0c0     corelib1:COREDLL.dll
 0002:000000c4       __imp___C_specific_handler 1000b0c4     corelib1:COREDLL.dll
 0002:000000c8       __imp_malloc               1000b0c8     corelib1:COREDLL.dll
 0002:000000cc       __imp_TerminateProcess     1000b0cc     coredll:COREDLL.dll
 0002:000000d0       \177COREDLL_NULL_THUNK_DATA 1000b0d0     coredll:COREDLL.dll
 0002:000000d4       __imp_DDKClockGetGatingMode 1000b0d4     cspddk:CSPDDK.dll
 0002:000000d8       __imp_DDKClockSetGatingMode 1000b0d8     cspddk:CSPDDK.dll
 0002:000000dc       __imp_DDKClockConfigBaud   1000b0dc     cspddk:CSPDDK.dll
 0002:000000e0       \177CSPDDK_NULL_THUNK_DATA 1000b0e0     cspddk:CSPDDK.dll
 0002:000000e8       dpCurSettings              1000b0e8     hwinit.obj
 0002:00000530       __security_cookie          1000b530     corelib0:seccinit.obj
 0002:00000534       __security_cookie_complement 1000b534     corelib0:seccinit.obj
 0002:00000538       m_hUSBClockGatingHandle    1000b538     i_usbclock.obj
 0002:0000053c       pUSBClkGating              1000b53c     i_usbclock.obj
 0002:00000540       g_pXVC                     1000b540     usb_xvc_mx25_topaz_v1:i_xvc.obj
 0002:00000544       gfsvaim                    1000b544     usb_xvc_mx25_topaz_v1:i_xvc.obj
 0002:00000548       _exitflag                  1000b548     corelib0:cexit.obj
 0002:0000054c       __onexitend                1000b54c     <common>
 0002:00000550       __onexitbegin              1000b550     <common>
 0002:00000554       g_pcsExit                  1000b554     <common>

 entry point at        0001:00008794

 Static symbols

 0001:000029bc       DumpDeviceState            100039bc f   hwinit.obj
 0001:00003890       ConfigOTGHost              10004890 f   hwinit.obj
 0001:00003c30       ConfigOTGClient            10004c30 f   hwinit.obj
 0001:00004168       BSPUsbXvrSetPhyPowerMode   10005168 f   hwinit.obj
 0001:00004848       USBClockSet                10005848 f   i_usbclock.obj
 0001:00004ea8       CeLogMsg                   10005ea8 f   usb_xvc_mx25_topaz_v1:i_xvc.obj
 0001:00005f6c       InitClock                  10006f6c f   usb_xvc_mx25_topaz_v1:i_xvc.obj
 0001:00005fa8       DeInitClock                10006fa8 f   usb_xvc_mx25_topaz_v1:i_xvc.obj
 0001:00005fe4       USBControllerRun           10006fe4 f   usb_xvc_mx25_topaz_v1:i_xvc.obj
 0001:00006304       USBControllerReset         10007304 f   usb_xvc_mx25_topaz_v1:i_xvc.obj
 0001:000076f8       PowerDown                  100086f8 f   usb_xvc_mx25_topaz_v1:i_xvc.obj
 0001:000078c8       PowerUp                    100088c8 f   usb_xvc_mx25_topaz_v1:i_xvc.obj
 0001:00007d28       GetStringParam             10008d28 f   usb_xvc_mx25_topaz_v1:i_registry.obj
 0001:00007f9c       GetDWordParam              10008f9c f   usb_xvc_mx25_topaz_v1:i_registry.obj
 0001:00008068       GetMultiDWordParam         10009068 f   usb_xvc_mx25_topaz_v1:i_registry.obj
 0001:00008354       GetBinParam                10009354 f   usb_xvc_mx25_topaz_v1:i_registry.obj
 0001:00008a38       doexit                     10009a38 f   corelib0:cexit.obj
 0001:00008cf4       lockexit                   10009cf4 f   corelib0:onexit.obj
 0001:00008d90       unlockexit                 10009d90 f   corelib0:onexit.obj
 0001:00008dbc       _onexit_nolock             10009dbc f   corelib0:onexit.obj
